:0E0000000AC0FECFFDCFFCCFFBCFFACFF9CF69
:10000E00F8CFF7CFF6CF0000F894EE27ECBBE5BFA4
:10001E00F8E1A4B7A77FA4BFF1BDE1BD8DE0A2E0DA
:10002E00ED938A95E9F780E4A0E6ED938A95E9F7DA
:10003E00E4E1F0E0C8953196802DC8953196902D6B
:10004E000097B9F0C8953196A02DC8953196B02D70
:10005E00C8953196102CC89531966E2F7F2FF02DA6
:10006E00E12DC89531960D920197D9F7E62FF72F0E
:10007E00E1CFEFE9EDBFC0E7D0E0B4C00A9300E0F6
:10008E00073118F4FCD00F5FFBCF73C0F7DF84E1AC
:10009E0095E00197F1F70895F1DF8CE39FE001976A
:1000AE00F1F708950A9300E0083058F4E981E17001
:1000BE0011F0F2DF01C0EADFE981E695E9830F5F17
:1000CE00F3CF08812296089511D100E010E00C358F
:1000DE00E1E01E0720F4D3D00F5F1F4FF8CFD8D02A
:1000EE0060C0C098B89A0895EFDFD2D0E1E0D5D0C5
:1000FE00EEEFD3D0E881D1D0E881E095CED0CCDF41
:10010E00EEE5F0E0CCD011C0DFDFC6DFECE8F0E0CA
:10011E00C6D00895E881E062E7B98DE08A95F1F7DF
:10012E00369A349BFECF349AE5B121960895DDD0F0
:10013E0010E020E000E00F3F30F4B4D08DE08A955F
:10014E00F1F70F5FF8CFAED0022FE02FD2D023966B
:10015E0008950A9300E0063058F4E9DFEE7FEF933E
:10016E00E6DFEE7FAF91EA1709F000E00F5FF3CF05
:10017E00DEDF09910895BAD0ECDF1E2F1C3D08F08A
:10018E000FEF1C3D08F402E41E3B08F40AE4183796
:10019E0008F40BE5103508F403E41E3108F403E00F
:1001AE00E02FABD00895B39907C0C19AE8E8F3E108
:1001BE0076D0B49B7ED001C07CD008957ED0E0E096
:1001CE00B499E1E0A1E08CD0E02121F072D0E0ED15
:1001DE00F7E065D0C1980895B49B02C0EFDF01C06F
:1001EE00E2DF0895E0E8E6BDE0E0E6BDE4B3E370EB
:1001FE00E4BBE4B3E4BBE0E2E7B9E2EAE6B9E3B1BB
:10020E00E87FE3B9C0986DDFC198B99A00E055D088
:10021E00E0E0C199E1E0A1E063D0E02109F0C198EE
:10022E00AADF4E2EEFEFE41591F34A925DDF6CDFFD
:10023E0000E0A1DFEF3F31F4EAE0F0E030D09BDFE9
:10024E00EF3FD9F0E2E0E415B9F0EAE4E415A1F0ED
:10025E005BDF0F5F033081F400E0E2E4E41521F48C
:10026E00E2E04E2EB9DF08C0EBE5E41529F4E9E52E
:10027E004E2E4A9239DF48DFDCCFC9CFFFCFC09A6E
:10028E0089E28A95F1F7C09889E28A95F1F7089587
:10029E00E6E0F0E0FA93EA9317C0EA9303CFFA93FD
:1002AE00EA9312C0E1E0EA9335DFF0E01E0F2F1F54
:1002BE000895E2E0EA9318DF27CFE0E0B399E1E09A
:1002CE00A1E00ED00E2E0895E991F991309639F0F5
:1002DE0088EE93E00197F1F7A8953197C9F7089545
:1002EE00EA17E1E009F0EE2708952A931A930A938C
:1002FE0008952A8119810881089509911991089507
:00000001FF
